S1230100BD0192CE02D6BD018FBDC00684DF81592708CE04F98D787EC0004F974397449700
S123012046CE03E58D69CE0041BDC012CE0042BDC012CE045A8D58BD01CB964597468601B3
S123014097479748BD02017D0049271CCE0041BDC012CE0042BDC012CE04DC8D32BDC006E8
S123016084DF814E27AC20B2BD024C7D00482718BD029D965297464F97489747CE05428DC6
S11501800E9652BDC00C20BCCE05548D0220A87EC00949
S1230192CE0020863FA700861EA701A706862DA702A7058633A703A7044FCE0001A72608ED
S12301B28C001326F88603A726088C001926F897594F974A9741974239BDC00680302F04DB
S12301D281062F07CE04948DB420EE974BBD01F02607CE04778DA620E0964B974539964B87
S12301F2270C81072708914627049B468107397F0049CE04B38D869646D6479B441997442F
S1230212CE0044BDC01296469B43974380122D167C00494D271F5D270ECE04D0BD018F865F
S1230232019B4219974239CE04C4BD018F86019B41199741395D27E120ED4F975397569FF8
S123025254CE000186269B4397579E5632A420A74B088C000726F586209740CE00069E5616
S1230272346D4B2613329A4036DF4A9E54BD01F02710964B9753200A7300403294403673AA
S123029200400974004026D69E5439BD02B7270096532702200CBD02B7974BBD01F027F626
S12302B2964B975239CE0003C609D459C1012705C1080C26010D7600587600590926E99616
S12302D2598407391B5B324A484921204C4554275320504C41592027313820574954482046
S12302F2412044494527210D0A594F552053544152542E2043484F4F534520414E59204E26
S1230312554D4245522C0D0A31205448525520362E204920444F204C494B45574953452C2C
S1230332204255542057450D0A43414E275420504C415920544845204E554D4245522054C8
S12303524845204F544845520D0A4A55535420504C415945442C204E4F522049545320446D
S12303724946464552454E43450D0A46524F4D20372E2054525920544F204D414B4520547C
S1230392484520544F54414C0D0A4F4620414C4C20594F555220504C415953204849542034
S12303B23138204F4E0D0A594F555220504C41592E0D0A0A524541445920544F20535441B6
S12303D252543F2028545950452059204F52204E2E29041B5B324A2020202020204549470E
S12303F2485445454E20574954482041204449450D0A0A2020202020202020202020202003
S12304122020202020202047414D455320574F4E0D0A20202020202020202020202020208E
S12304322020202020202020594F55204D450D0A544F54414C204953203030202020202080
S123045220202020202020040D0A0A2020202020202020594F555220464952535420504CCE
S123047241593F20040D0A494C4C4547414C20504C4159212054525920414E4F5448455291
S12304922E040D0A494E56414C494420504C41592120504C41592031205448525520362EF1
S12304B2041B5B480A0A0A0A544F54414C20495320042020594F552057494E212004202008
S12304D2492057494E21202020040A0D0A1B5B4A4E45572047414D453F2028275927204F88
S12304F25220274E2729040D0A5448414E4B5320464F5220504C4159494E472E20484F505B
S12305124520594F550D0A454E4A4F594544204954204153204D55434820415320492E0D28
S12305320A53454520594F55204C4154455221040A0D0A1B5B4A4D5920504C41592049534B
S115055220040A0A2E20594F555220504C41593F200405
S9030000FC
